:020000040000FA
:020000001F28B7
:08000800F000030EF1000A08EC
:10001000F20083128B181D28283081000B11F40385
:10002000F30B16281330F300F503761472088A00D8
:10003000710E8300F00E700E09008B101628073029
:100040009F000A30F70058208316E0308500FF300B
:100050008600073081008312013090008B138B15CE
:1000600086080B106300000086080B108B11061E1B
:100070003728283081001330F3000530F500F601F1
:100080000B11A0308B00F7010314F70D5820761CDC
:100090004728F6017508031D44280E08F4000310D4
:1000A000F40C7408031D51288B13F70158202E28D7
:0800B00077081F3A85000800E3
:02400E00103F61
:00000001FF
